:100000008D2E83120313B300B4011130B5001528EF
:1000100083120313B40DB60D3308340236180314DB
:10002000031C152883120313B40083120313B10DAC
:10003000B20DB50B08283108080083120313B30072
:10004000B4011030B50083120313B10DB20DB40D1D
:10005000B60D3308340236180314031C32288312F9
:100060000313B40083120313B50B232834080800CC
:1000700083120313A3000310230CA5000630AC0069
:10008000AD015C2083120313A4018312031325081E
:100090002402031851280000000000000000A40AF8
:1000A0004528080083120313B10031089900831614
:1000B0000313981C5728080083120313AE01023063
:1000C000831681000230831281000D3083120313E6
:1000D000AE078312031301082E06031D692883123D
:1000E0000313AC032C0A0319AD032C082D04031DC4
:1000F0006528080083120313A901023083168100CA
:100100000230831281007D3083120313A90783120A
:10011000031301082906031D872883120313A7036D
:10012000270A0319A80327082804031D83280800A9
:1001300083120313AA00F0302A05AB002B0E0F39EF
:10014000AB000A302B020318A8283030AB07AE28CA
:100150000A3083120313AB024130AB07831203133F
:100160002B08D7000F302A05AB000A302B020318EA
:10017000BC283030AB07C2280A3083120313AB020D
:100180004130AB07831203132B08D80008008312F9
:1001900003132708B1002808B2000A301D2083127B
:1001A0000313AD002708B1002808B2000A3001206F
:1001B000831203133108AE003208AF002E08B100DD
:1001C0002F08B2000A301D2083120313AC00270849
:1001D000B1002808B20064300120831203133108F3
:1001E000AE003208AF002E08B1002F08B2000A306E
:1001F0001D2083120313AB002E08B1002F08B2009C
:100200000A300120831203133108B0003008B10016
:10021000B2010A301D2083120313AA002E08B10078
:100220002F08B20064300120831203133108B0009C
:100230003008A900CA010530831203134A020318CB
:100240002C2929304A0784008313303000075220BC
:1002500083120313CA0A1B29080083120313A30085
:100260002308B100B2010A301D2083120313A60037
:100270002308B100B2010A300120831203133108B0
:10028000A7002708B100B2010A301D208312031312
:10029000A5002308B100B2016430012083120313CA
:1002A0003108A7002708A400CA01033083120313F2
:1002B0004A020318662924304A0784008313303029
:1002C0000007522083120313CA0A5529080083121B
:1002D0000313C001C101C201C301C401C501C601AC
:1002E000C7010800831203133C1C7F29B9013E0893
:1002F000A7002C14A12183120313B80089298312AB
:100300000313B8013E08A7002C10A1218312031388
:10031000B90083120313BC1C9629BA013F08A70039
:100320002C14A12183120313BB00A02983120313F1
:10033000BB013F08A7002C10A12183120313BA00B0
:100340000800831203132C1CAC292709A800A9015B
:10035000A80A0319A90AB129831203132708A800C0
:10036000A901033083120313AD000310831203139A
:10037000A80DA90DAD0BB5292808B1002908B200B8
:100380000F300120831203133108AA003208AB009A
:100390002A080800831203135408C8005508BE0039
:1003A0005608BF00BC11C81BBC153C11481B3C15AE
:1003B000BC10C81ABC143C10481A3C14BC12481992
:1003C000BC163C13C8183C173C1248183C160800D1
:1003D00083120313861BF529061BF029B701002A97
:1003E0000A3083120313B700002A83120313061B7B
:1003F000FC290530B700002A0F3083120313B70021
:1004000083120313B708031D2A2ABE080319122AF0
:100410003C1C0D2A85170513162A83120313851316
:100420000517162A8312031385130513831203136A
:10043000BF080319252ABC1C202A05148510562A3A
:100440008312031305108514562A83120313051013
:100450008510562A83120313390837020318332AEA
:1004600005178513402A831203133808370203182F
:100470003C2A85170513402A83120313851305139D
:10048000831203133A0837020318492A851405100A
:10049000562A831203133B0837020318522A051405
:1004A0008510562A83120313851005100800831245
:1004B0000313A700D901831203132C14AC10492491
:1004C0008312031327082924831203132910031806
:1004D00029140330AC00AD015C20831203132C10EF
:1004E000AC104924831203132C10AC14492483123A
:1004F0000313861E772A83120313861A7B2A83121C
:1005000003132C1027182C14AC1449248312031342
:10051000861E862A83120313861A8A2A83120313DD
:100520002C10A7182C14AC14492483120313861E14
:10053000952A83120313861A992A831203132C1007
:1005400027192C14AC14492483120313861EA42AE1
:1005500083120313861AA82A831203132C10A719D7
:100560002C14AC14492483120313861EB32A83125D
:100570000313861AB72A831203132C10271A2C147C
:10058000AC14492483120313861EC22A8312031358
:10059000861AC62A831203132C10A71A2C14AC1423
:1005A000492483120313861ED12A83120313861A49
:1005B000D52A831203132C10271B2C14AC144924A6
:1005C00083120313861EE02A83120313861AE42A79
:1005D000831203132C10A71B2C14AC144924831270
:1005E0000313861EEF2A83120313861AF32A83123B
:1005F00003132C1029182C14AC1449248312031350
:10060000861EFE2A83120313861A022B83120313FB
:100610002C14AC14492483120313861A0B2B86194D
:100620000B2B83120313861E112B861D112B2523E2
:10063000031C172B831203135908982083120313EA
:100640005908FA3A031D5B2A080083120313AB0111
:100650002C14AC104924013083120313AC00AD01FB
:100660005C20831203132C14AC144924831203134B
:10067000861E362B83120313AA01643083120313E0
:100680002A020318532B861A472B861D532B8312DD
:1006900003132A08633A031D4F2B0310080083122B
:1006A0000313AA0A3D2B83120313861E532B8312B6
:1006B0000313861A572B831203132B1086192B143E
:1006C00083120313861E602B83120313861A642B76
:1006D00083120313AB108619AB1483120313861E07
:1006E0006D2B83120313861A712B831203132B11A4
:1006F00086192B1583120313861E7A2B831203137C
:10070000861A7E2B83120313AB118619AB15831245
:100710000313861E872B83120313861A8B2B8312D7
:1007200003132B1286192B1683120313861E942B88
:1007300083120313861A982B83120313AB128619A4
:10074000AB1683120313861EA12B83120313861A82
:10075000A52B831203132B1386192B178312031354
:10076000861EAE2B83120313861AB22B8312031339
:10077000AB138619AB1783120313861EBB2B831290
:100780000313861ABF2B83120313861EC32B8312F7
:100790000313861AC72B831203132B08D9000314E3
:1007A000080083120313D401D501D601CA01053014
:1007B000831203134A020318EC2B25230318EC2B96
:1007C000831203134A08043A031DE82B03100800A0
:1007D00083120313CA0AD72B831203135908D400B8
:1007E00025230318F52B031008008312031359085F
:1007F000D50025230318FE2B0310080083120313D2
:100800005908D60003140800043083120313CB00E8
:10081000FF3057222523031C0A2C83120313590887
:10082000A0002523031C112C831203132008AA3ACD
:10083000031D212CF33057220A305722F43057225F
:10084000282C831203132008FC3A031901340234C4
:10085000003483120313AA002D1401302A18AD06A8
:100860000130AA18AD0601302A19AD060130AA19C7
:10087000AD0601302A1AAD060130AA1AAD060130C4
:100880002A1BAD060130AA1BAD0603102D18031458
:100890000800831203132C1C502C83168615552C2C
:1008A0008312031386118316861183120313AC1C63
:1008B0005C2C83168616612C831203138612831612
:1008C0008612080083120313C9014910051949143F
:1008D000C9108519C91406187F2C4B08023A031950
:1008E0007F2CE83057222523031C732C013057221C
:1008F0002523031C782C023083120313CB008312B0
:100900000313061C952C4B08043A0319952CE83068
:1009100057222523031C892C023057222523031C30
:100920008E2C043083120313CB00080083120313B0
:10093000C908031D0A2DA1010330831203132102EC
:100940000318C52CA0010A308312031320020318D8
:10095000C12CD123031CB32CCA217221E8210A30F7
:1009600083120313A000831203132008093A031D06
:10097000BD2C851005108513051383120313A00ADF
:10098000A32C83120313A10A9C2C83120313051AB0
:10099000082D851CCE2C31305220D02C30305220E6
:1009A00083120313051CD72C31305220D92C303040
:1009B000522083120313851FE02C31305220E22C89
:1009C0003030522083120313051FE92C313052209E
:1009D000EB2C30305220831203133C1EF22C3130AA
:1009E0005220F42C3030522083120313BC1EFB2CF7
:1009F00031305220FD2C30305220831203133C1F23
:100A0000042D31305220062D303052202C3052200F
:100A10006224962C080083120313490B9B2DA0011E
:100A20000A3083120313200203186A2DD123031CFA
:100A30001B2DCA2172218030831203133B0203183D
:100A4000252D80303B07A100292DFF308312031391
:100A5000A1008030831203133A020318322D3A08A2
:100A6000A102352D83120313A101831203138514F0
:100A70000514210838208312031385100510D12393
:100A8000031C442DCA2172218030831203133802C3
:100A900003184E2D80303807A200522DFF308312EC
:100AA0000313A200803083120313390203185B2D55
:100AB0003908A2025E2D83120313A20183120313CD
:100AC0008517051722083820831203138513051391
:100AD000A00A102D83120313051A992D3A082D210F
:100AE000831203133B082D218312031338082D2191
:100AF0008312031339082D21831203133C1E832D07
:100B000031305220852D3030522083120313BC1E09
:100B10008C2D313052208E2D303052208312031311
:100B20003C1F952D31305220972D303052202C30E3
:100B3000522062240B2D0800831203134908A000E1
:100B40006721831203134908023A0319AB2D4908A0
:100B5000033A031D8C2E8312031349082006031940
:100B6000B42D4908A000672183120313A610261193
:100B7000A2010A3083120313220203183A2ED12352
:100B8000031C242E83120313A618212ECA218312BC
:100B90000313A3010A308312031323020318212E27
:100BA000D123031C1D2E8312031326191A2ECA21CA
:100BB0007221E821831203134108A1003A08C007FB
:100BC0000318C10A210841020318EA2D6721831284
:100BD00003132614831203134308A1003B08C20722
:100BE0000318C30A210843020318FA2D6721831250
:100BF00003132614831203134508A1003808C40701
:100C00000318C50A2108450203180A2E672183121A
:100C100003132614831203134708A1003908C607DB
:100C20000318C70A2108470203181A2E67218312E6
:100C30000313261483120313261583120313A30A26
:100C4000CA2D83120313A614831203132208093A30
:100C5000031D362E2619362E6F30A700A8017A20E4
:100C600083120313851005108513051383120313D4
:100C7000A20AB92D83120313051A8A2E261C512E9F
:100C8000CA011430831203134A0203184D2E39305F
:100C9000522083120313CA0A412E83120313261013
:100CA0006D2E831203134008A7004108A800C72037
:100CB000831203134208A7004308A800C720831229
:100CC00003134408A7004508A800C7208312031394
:100CD0004608A7004708A800C720831203133C1E3C
:100CE000742E31305220762E30305220831203136E
:100CF000BC1E7D2E313052207F2E30305220831288
:100D000003133C1F862E31305220882E3030522063
:100D10002C3052206224A12D0800073083120313C7
:100D20009F0085013C308316850083128601FF30C9
:100D30008316860019309900243098009030831271
:100D40009800831681130424003A031DA32E8312F6
:100D500003133C12BC123C13622483120313490890
:100D60000319BC2E013A0319BE2E033A0319C02EF3
:100D7000013A0319C22EAC2E9624AC2E0B25AC2EB4
:080D80009C25AC2E9C25AC2E35
:02400E00703E02
:00000001FF
